 npt

 Timestamp is 6710e050 (Thu Oct 17 10:00:48 2024)

 Preferred load address is 10000000

 Start         Length     Name                   Class
 0001:00000000 00001721H .text$mn                CODE
 0002:00000000 000000b4H .idata$5                DATA
 0002:000000b4 00000008H .00cfg                  DATA
 0002:000000bc 00000004H .CRT$XCA                DATA
 0002:000000c0 00000004H .CRT$XCZ                DATA
 0002:000000c4 00000004H .CRT$XIA                DATA
 0002:000000c8 00000004H .CRT$XIZ                DATA
 0002:000000cc 00000004H .CRT$XPA                DATA
 0002:000000d0 00000004H .CRT$XPZ                DATA
 0002:000000d4 00000004H .CRT$XTA                DATA
 0002:000000d8 00000008H .CRT$XTZ                DATA
 0002:000000dc 00000000H .gfids$y                DATA
 0002:000000e0 000002e0H .rdata                  DATA
 0002:000003c0 00000000H .rdata$CastGuardVftablesA DATA
 0002:000003c0 00000000H .rdata$CastGuardVftablesC DATA
 0002:000003c0 00000004H .rdata$sxdata           DATA
 0002:000003c4 0000005cH .rdata$voltmd           DATA
 0002:00000420 000002e4H .rdata$zzzdbg           DATA
 0002:00000704 00000004H .rtc$IAA                DATA
 0002:00000708 00000004H .rtc$IZZ                DATA
 0002:0000070c 00000004H .rtc$TAA                DATA
 0002:00000710 00000008H .rtc$TZZ                DATA
 0002:00000718 00000088H .xdata$x                DATA
 0002:000007a0 00000060H .edata                  DATA
 0002:00000800 0000008cH .idata$2                DATA
 0002:0000088c 00000014H .idata$3                DATA
 0002:000008a0 000000b4H .idata$4                DATA
 0002:00000954 000003a6H .idata$6                DATA
 0003:00000000 00000018H .data                   DATA
 0003:00000018 00000374H .bss                    DATA
 0004:00000000 00000060H .rsrc$01                DATA
 0004:00000060 00000308H .rsrc$02                DATA

  Address         Publics by Value              Rva+Base       Lib:Object

 0000:00000000       ___AbsoluteZero            00000000     <absolute>
 0000:00000000       ___arm64x_extra_rfe_table  00000000     <absolute>
 0000:00000000       ___arm64x_extra_rfe_table_size 00000000     <absolute>
 0000:00000000       ___arm64x_native_entrypoint 00000000     <absolute>
 0000:00000000       ___arm64x_redirection_metadata 00000000     <absolute>
 0000:00000000       ___arm64x_redirection_metadata_count 00000000     <absolute>
 0000:00000000       ___dynamic_value_reloc_table 00000000     <absolute>
 0000:00000000       ___enclave_config          00000000     <absolute>
 0000:00000000       ___guard_check_icall_a64n_fptr 00000000     <absolute>
 0000:00000000       ___guard_eh_cont_count     00000000     <absolute>
 0000:00000000       ___guard_eh_cont_table     00000000     <absolute>
 0000:00000000       ___guard_fids_count        00000000     <absolute>
 0000:00000000       ___guard_fids_table        00000000     <absolute>
 0000:00000000       ___guard_iat_count         00000000     <absolute>
 0000:00000000       ___guard_iat_table         00000000     <absolute>
 0000:00000000       ___guard_longjmp_count     00000000     <absolute>
 0000:00000000       ___guard_longjmp_table     00000000     <absolute>
 0000:00000000       ___hybrid_auxiliary_delayload_iat 00000000     <absolute>
 0000:00000000       ___hybrid_auxiliary_delayload_iat_copy 00000000     <absolute>
 0000:00000000       ___hybrid_auxiliary_iat    00000000     <absolute>
 0000:00000000       ___hybrid_auxiliary_iat_copy 00000000     <absolute>
 0000:00000000       ___hybrid_code_map         00000000     <absolute>
 0000:00000000       ___hybrid_code_map_count   00000000     <absolute>
 0000:00000000       ___hybrid_image_info_bitfield 00000000     <absolute>
 0000:00000000       ___x64_code_ranges_to_entry_points 00000000     <absolute>
 0000:00000000       ___x64_code_ranges_to_entry_points_count 00000000     <absolute>
 0000:00000001       ___safe_se_handler_count   00000001     <absolute>
 0000:00000100       ___guard_flags             00000100     <absolute>
 0000:00000000       ___ImageBase               10000000     <linker-defined>
 0001:00000000       ___local_stdio_printf_options 10001000 f i npt.obj
 0001:00000006       __vfprintf_l               10001006 f i npt.obj
 0001:0000002a       _fprintf                   1000102a f i npt.obj
 0001:00000042       _nptInitialize@12          10001042 f   npt.obj
 0001:00000116       _nptTerminate@8            10001116 f   npt.obj
 0001:00000137       _utf16ToUtf8m@20           10001137 f   utf.obj
 0001:00000288       _utf16ToUtf8s@20           10001288 f   utf.obj
 0001:0000028e       _utf8ToUtf16@20            1000128e f   utf.obj
 0001:00000368       _utf8mToUtf8s@20           10001368 f   utf.obj
 0001:00000508       _utf8mToUtf8sLength@12     10001508 f   utf.obj
 0001:000005e8       _utf8sToUtf8m@20           100015e8 f   utf.obj
 0001:00000718       _utf8sToUtf8mLength@12     10001718 f   utf.obj
 0001:000007da       _utfError                  100017da f   utf.obj
 0001:00000892       _utf8FromPlatform@20       10001892 f   utf_md.obj
 0001:00000918       _utf8ToPlatform@20         10001918 f   utf_md.obj
 0001:0000099e       _utfInitialize@4           1000199e f   utf_md.obj
 0001:00000a02       _utfTerminate@8            10001a02 f   utf_md.obj
 0001:00000a10       @__security_check_cookie@4 10001a10 f   MSVCRT:secchk.obj
 0001:00000d5e       __DllMainCRTStartup@12     10001d5e f   MSVCRT:dll_dllmain.obj
 0001:00000d81       ___raise_securityfailure   10001d81 f   MSVCRT:gs_report.obj
 0001:00000da9       ___report_gsfailure        10001da9 f   MSVCRT:gs_report.obj
 0001:00000ef0       ___security_init_cookie    10001ef0 f   MSVCRT:gs_support.obj
 0001:00000f3b       _DllMain@12                10001f3b f   MSVCRT:dll_dllmain_stub.obj
 0001:00000f5d       ?__scrt_initialize_type_info@@YAXXZ 10001f5d f   MSVCRT:tncleanup.obj
 0001:00000f69       ?__scrt_uninitialize_type_info@@YAXXZ 10001f69 f   MSVCRT:tncleanup.obj
 0001:00000f75       ___local_stdio_scanf_options 10001f75 f i MSVCRT:default_local_stdio_options.obj
 0001:00000f7b       ___scrt_initialize_default_local_stdio_options 10001f7b f   MSVCRT:default_local_stdio_options.obj
 0001:00000fdc       ___scrt_acquire_startup_lock 10001fdc f   MSVCRT:utility.obj
 0001:0000100e       ___scrt_dllmain_after_initialize_c 1000200e f   MSVCRT:utility.obj
 0001:00001039       ___scrt_dllmain_before_initialize_c 10002039 f   MSVCRT:utility.obj
 0001:00001047       ___scrt_dllmain_crt_thread_attach 10002047 f   MSVCRT:utility.obj
 0001:00001066       ___scrt_dllmain_crt_thread_detach 10002066 f   MSVCRT:utility.obj
 0001:00001073       ___scrt_dllmain_exception_filter 10002073 f   MSVCRT:utility.obj
 0001:000010a7       ___scrt_dllmain_uninitialize_c 100020a7 f   MSVCRT:utility.obj
 0001:000010ca       ___scrt_dllmain_uninitialize_critical 100020ca f   MSVCRT:utility.obj
 0001:000010d7       ___scrt_initialize_crt     100020d7 f   MSVCRT:utility.obj
 0001:00001110       ___scrt_initialize_onexit_tables 10002110 f   MSVCRT:utility.obj
 0001:00001197       ___scrt_is_nonwritable_in_current_image 10002197 f   MSVCRT:utility.obj
 0001:0000122b       ___scrt_release_startup_lock 1000222b f   MSVCRT:utility.obj
 0001:00001248       ___scrt_uninitialize_crt   10002248 f   MSVCRT:utility.obj
 0001:00001270       ___scrt_get_dyn_tls_init_callback 10002270 f   MSVCRT:dyn_tls_init.obj
 0001:00001276       ___scrt_fastfail           10002276 f   MSVCRT:utility_desktop.obj
 0001:00001391       __crt_debugger_hook        10002391 f   MSVCRT:utility_desktop.obj
 0001:00001399       __RTC_Initialize           10002399 f   MSVCRT:initsect.obj
 0001:000013c5       __RTC_Terminate            100023c5 f   MSVCRT:initsect.obj
 0001:00001400       __SEH_prolog4              10002400 f   MSVCRT:sehprolg4.obj
 0001:00001445       __except_handler4          10002445 f   MSVCRT:chandler4gs.obj
 0001:00001474       @_guard_check_icall_nop@4  10002474 f i MSVCRT:guard_support.obj
 0001:00001477       ___isa_available_init      10002477 f   MSVCRT:cpu_disp.obj
 0001:0000164b       __get_startup_argv_mode    1000264b f   MSVCRT:argv_mode.obj
 0001:0000164f       ___scrt_is_ucrt_dll_in_use 1000264f f   MSVCRT:ucrt_detection.obj
 0001:0000165b       ___std_type_info_destroy_list 1000265b f   vcruntime:VCRUNTIME140.dll
 0001:00001661       _memset                    10002661 f   vcruntime:VCRUNTIME140.dll
 0001:00001667       __except_handler4_common   10002667 f   vcruntime:VCRUNTIME140.dll
 0001:0000166d       _strcmp                    1000266d f   ucrt:api-ms-win-crt-string-l1-1-0.dll
 0001:00001673       __initterm                 10002673 f   ucrt:api-ms-win-crt-runtime-l1-1-0.dll
 0001:00001679       __initterm_e               10002679 f   ucrt:api-ms-win-crt-runtime-l1-1-0.dll
 0001:0000167f       __seh_filter_dll           1000267f f   ucrt:api-ms-win-crt-runtime-l1-1-0.dll
 0001:00001685       __configure_narrow_argv    10002685 f   ucrt:api-ms-win-crt-runtime-l1-1-0.dll
 0001:0000168b       __initialize_narrow_environment 1000268b f   ucrt:api-ms-win-crt-runtime-l1-1-0.dll
 0001:00001691       __initialize_onexit_table  10002691 f   ucrt:api-ms-win-crt-runtime-l1-1-0.dll
 0001:00001697       __execute_onexit_table     10002697 f   ucrt:api-ms-win-crt-runtime-l1-1-0.dll
 0001:0000169d       __cexit                    1000269d f   ucrt:api-ms-win-crt-runtime-l1-1-0.dll
 0001:000016a3       ___acrt_initialize         100026a3 f   MSVCRT:ucrt_stubs.obj
 0001:000016a3       ___acrt_thread_attach      100026a3 f   MSVCRT:ucrt_stubs.obj
 0001:000016a3       ___acrt_thread_detach      100026a3 f   MSVCRT:ucrt_stubs.obj
 0001:000016a3       ___acrt_uninitialize       100026a3 f   MSVCRT:ucrt_stubs.obj
 0001:000016a3       ___acrt_uninitialize_critical 100026a3 f   MSVCRT:ucrt_stubs.obj
 0001:000016a3       ___scrt_stub_for_acrt_initialize 100026a3 f   MSVCRT:ucrt_stubs.obj
 0001:000016a3       ___scrt_stub_for_acrt_thread_attach 100026a3 f   MSVCRT:ucrt_stubs.obj
 0001:000016a3       ___scrt_stub_for_acrt_thread_detach 100026a3 f   MSVCRT:ucrt_stubs.obj
 0001:000016a3       ___scrt_stub_for_acrt_uninitialize 100026a3 f   MSVCRT:ucrt_stubs.obj
 0001:000016a3       ___scrt_stub_for_acrt_uninitialize_critical 100026a3 f   MSVCRT:ucrt_stubs.obj
 0001:000016a3       ___vcrt_initialize         100026a3 f   MSVCRT:ucrt_stubs.obj
 0001:000016a3       ___vcrt_thread_attach      100026a3 f   MSVCRT:ucrt_stubs.obj
 0001:000016a3       ___vcrt_thread_detach      100026a3 f   MSVCRT:ucrt_stubs.obj
 0001:000016a3       ___vcrt_uninitialize       100026a3 f   MSVCRT:ucrt_stubs.obj
 0001:000016a3       ___vcrt_uninitialize_critical 100026a3 f   MSVCRT:ucrt_stubs.obj
 0001:000016a6       ___scrt_stub_for_is_c_termination_complete 100026a6 f   MSVCRT:ucrt_stubs.obj
 0001:000016a6       __is_c_termination_complete 100026a6 f   MSVCRT:ucrt_stubs.obj
 0001:000016a9       __filter_x86_sse2_floating_point_exception 100026a9 f   MSVCRT:x86_exception_filter.obj
 0001:000016a9       __filter_x86_sse2_floating_point_exception_default 100026a9 f   MSVCRT:x86_exception_filter.obj
 0002:00000000       __imp__MultiByteToWideChar@24 10003000     kernel32:KERNEL32.dll
 0002:00000004       __imp__WideCharToMultiByte@32 10003004     kernel32:KERNEL32.dll
 0002:00000008       __imp__GetACP@0            10003008     kernel32:KERNEL32.dll
 0002:0000000c       __imp__GetLocaleInfoA@16   1000300c     kernel32:KERNEL32.dll
 0002:00000010       __imp__GetUserDefaultLCID@0 10003010     kernel32:KERNEL32.dll
 0002:00000014       __imp__UnhandledExceptionFilter@4 10003014     kernel32:KERNEL32.dll
 0002:00000018       __imp__SetUnhandledExceptionFilter@4 10003018     kernel32:KERNEL32.dll
 0002:0000001c       __imp__GetCurrentProcess@0 1000301c     kernel32:KERNEL32.dll
 0002:00000020       __imp__TerminateProcess@8  10003020     kernel32:KERNEL32.dll
 0002:00000024       __imp__IsProcessorFeaturePresent@4 10003024     kernel32:KERNEL32.dll
 0002:00000028       __imp__QueryPerformanceCounter@4 10003028     kernel32:KERNEL32.dll
 0002:0000002c       __imp__GetCurrentProcessId@0 1000302c     kernel32:KERNEL32.dll
 0002:00000030       __imp__GetCurrentThreadId@0 10003030     kernel32:KERNEL32.dll
 0002:00000034       __imp__GetSystemTimeAsFileTime@4 10003034     kernel32:KERNEL32.dll
 0002:00000038       __imp__DisableThreadLibraryCalls@4 10003038     kernel32:KERNEL32.dll
 0002:0000003c       __imp__InitializeSListHead@4 1000303c     kernel32:KERNEL32.dll
 0002:00000040       __imp__IsDebuggerPresent@0 10003040     kernel32:KERNEL32.dll
 0002:00000044       \177KERNEL32_NULL_THUNK_DATA 10003044     kernel32:KERNEL32.dll
 0002:00000048       __imp____std_type_info_destroy_list 10003048     vcruntime:VCRUNTIME140.dll
 0002:0000004c       __imp__memset              1000304c     vcruntime:VCRUNTIME140.dll
 0002:00000050       __imp___except_handler4_common 10003050     vcruntime:VCRUNTIME140.dll
 0002:00000054       \177VCRUNTIME140_NULL_THUNK_DATA 10003054     vcruntime:VCRUNTIME140.dll
 0002:00000058       __imp__atoi                10003058     ucrt:api-ms-win-crt-convert-l1-1-0.dll
 0002:0000005c       \177api-ms-win-crt-convert-l1-1-0_NULL_THUNK_DATA 1000305c     ucrt:api-ms-win-crt-convert-l1-1-0.dll
 0002:00000060       __imp__calloc              10003060     ucrt:api-ms-win-crt-heap-l1-1-0.dll
 0002:00000064       __imp__free                10003064     ucrt:api-ms-win-crt-heap-l1-1-0.dll
 0002:00000068       __imp__malloc              10003068     ucrt:api-ms-win-crt-heap-l1-1-0.dll
 0002:0000006c       \177api-ms-win-crt-heap-l1-1-0_NULL_THUNK_DATA 1000306c     ucrt:api-ms-win-crt-heap-l1-1-0.dll
 0002:00000070       __imp__abort               10003070     ucrt:api-ms-win-crt-runtime-l1-1-0.dll
 0002:00000074       __imp__exit                10003074     ucrt:api-ms-win-crt-runtime-l1-1-0.dll
 0002:00000078       __imp___initterm           10003078     ucrt:api-ms-win-crt-runtime-l1-1-0.dll
 0002:0000007c       __imp___initterm_e         1000307c     ucrt:api-ms-win-crt-runtime-l1-1-0.dll
 0002:00000080       __imp___seh_filter_dll     10003080     ucrt:api-ms-win-crt-runtime-l1-1-0.dll
 0002:00000084       __imp___configure_narrow_argv 10003084     ucrt:api-ms-win-crt-runtime-l1-1-0.dll
 0002:00000088       __imp___initialize_narrow_environment 10003088     ucrt:api-ms-win-crt-runtime-l1-1-0.dll
 0002:0000008c       __imp___cexit              1000308c     ucrt:api-ms-win-crt-runtime-l1-1-0.dll
 0002:00000090       __imp___execute_onexit_table 10003090     ucrt:api-ms-win-crt-runtime-l1-1-0.dll
 0002:00000094       __imp___initialize_onexit_table 10003094     ucrt:api-ms-win-crt-runtime-l1-1-0.dll
 0002:00000098       \177api-ms-win-crt-runtime-l1-1-0_NULL_THUNK_DATA 10003098     ucrt:api-ms-win-crt-runtime-l1-1-0.dll
 0002:0000009c       __imp____stdio_common_vfprintf 1000309c     ucrt:api-ms-win-crt-stdio-l1-1-0.dll
 0002:000000a0       __imp____acrt_iob_func     100030a0     ucrt:api-ms-win-crt-stdio-l1-1-0.dll
 0002:000000a4       \177api-ms-win-crt-stdio-l1-1-0_NULL_THUNK_DATA 100030a4     ucrt:api-ms-win-crt-stdio-l1-1-0.dll
 0002:000000a8       __imp___strdup             100030a8     ucrt:api-ms-win-crt-string-l1-1-0.dll
 0002:000000a8       __imp__strdup              100030a8     ucrt:api-ms-win-crt-string-l1-1-0.dll
 0002:000000ac       __imp__strcmp              100030ac     ucrt:api-ms-win-crt-string-l1-1-0.dll
 0002:000000b0       \177api-ms-win-crt-string-l1-1-0_NULL_THUNK_DATA 100030b0     ucrt:api-ms-win-crt-string-l1-1-0.dll
 0002:000000b4       ___guard_check_icall_fptr  100030b4     MSVCRT:guard_support.obj
 0002:000000b8       ___castguard_check_failure_os_handled_fptr 100030b8     MSVCRT:guard_support.obj
 0002:000000bc       ___xc_a                    100030bc     MSVCRT:initializers.obj
 0002:000000c0       ___xc_z                    100030c0     MSVCRT:initializers.obj
 0002:000000c4       ___xi_a                    100030c4     MSVCRT:initializers.obj
 0002:000000c8       ___xi_z                    100030c8     MSVCRT:initializers.obj
 0002:000000cc       ___xp_a                    100030cc     MSVCRT:initializers.obj
 0002:000000d0       ___xp_z                    100030d0     MSVCRT:initializers.obj
 0002:000000d4       ___xt_a                    100030d4     MSVCRT:initializers.obj
 0002:000000d8       ___xt_z                    100030d8     MSVCRT:initializers.obj
 0002:000000e0       ??_C@_05CJAIGNCM@0?40?40@  100030e0     npt.obj
 0002:000000e8       ??_C@_0BK@LLKHEIF@NPT?5version?5doesn?8t?5match@ 100030e8     npt.obj
 0002:00000104       ??_C@_0P@KEJEBKCF@NPT?5ERROR?3?5?$CFs?6@ 10003104     npt.obj
 0002:00000114       ??_C@_0CJ@CPPDLDHE@Cannot?5allocate?5calloc?5space?5fo@ 10003114     npt.obj
 0002:00000140       ??_C@_0BJ@NDKKCKOJ@UTF?5ERROR?5?$FL?$CC?$CFs?$CC?3?$CFd?$FN?3?5?$CFs?6@ 10003140     utf.obj
 0002:0000015c       ??_C@_0BC@FAJHJFKN@ASSERT?5ERROR?5utf8@ 1000315c     utf.obj
 0002:00000170       ??_C@_05HLMOHPHA@utf?4c@   10003170     utf.obj
 0002:00000178       ??_C@_0BE@EHOOKJPG@ASSERT?5ERROR?5len?$DO?$DN0@ 10003178     utf.obj
 0002:0000018c       ??_C@_0BE@MONHEHKE@ASSERT?5ERROR?5output@ 1000318c     utf.obj
 0002:000001a0       ??_C@_0BM@BJKMEOOG@ASSERT?5ERROR?5outputMaxLen?$DO0@ 100031a0     utf.obj
 0002:000001bc       ??_C@_0BD@COPKOCDK@ASSERT?5ERROR?5utf16@ 100031bc     utf.obj
 0002:000001d0       ??_C@_0BH@PGKNPGMC@ASSERT?5ERROR?5i?$DN?$DNlength@ 100031d0     utf.obj
 0002:000001e8       ??_C@_0BK@HADMOKCE@ASSERT?5ERROR?5j?$DN?$DNnewLength@ 100031e8     utf.obj
 0002:00000204       ??_C@_0BN@ILDOBJEF@Can?8t?5get?5WIDE?5string?5length@ 10003204     utf_md.obj
 0002:00000224       ??_C@_08DHIDLBHK@utf_md?4c@ 10003224     utf_md.obj
 0002:00000230       ??_C@_0BJ@LFBNLHDK@Can?8t?5malloc?$CI?$CJ?5any?5space@ 10003230     utf_md.obj
 0002:0000024c       ??_C@_0BG@OELEGHKP@Can?8t?5get?5WIDE?5string@ 1000324c     utf_md.obj
 0002:00000264       ??_C@_0CI@EJHCPIBO@Can?8t?5convert?5WIDE?5string?5to?5mu@ 10003264     utf_md.obj
 0002:0000028c       __pDefaultRawDllMain       1000328c     MSVCRT:dll_dllmain.obj
 0002:0000028c       __pRawDllMain              1000328c     MSVCRT:dll_dllmain.obj
 0002:00000298       __load_config_used         10003298     MSVCRT:loadcfg.obj
 0002:000003c0       ___safe_se_handler_table   100033c0     <linker-defined>
 0002:000003c4       ___volatile_metadata       100033c4     <linker-defined>
 0002:00000704       ___rtc_iaa                 10003704     MSVCRT:initsect.obj
 0002:00000708       ___rtc_izz                 10003708     MSVCRT:initsect.obj
 0002:0000070c       ___rtc_taa                 1000370c     MSVCRT:initsect.obj
 0002:00000710       ___rtc_tzz                 10003710     MSVCRT:initsect.obj
 0002:00000800       __IMPORT_DESCRIPTOR_KERNEL32 10003800     kernel32:KERNEL32.dll
 0002:00000814       __IMPORT_DESCRIPTOR_VCRUNTIME140 10003814     vcruntime:VCRUNTIME140.dll
 0002:00000828       __IMPORT_DESCRIPTOR_api-ms-win-crt-stdio-l1-1-0 10003828     ucrt:api-ms-win-crt-stdio-l1-1-0.dll
 0002:0000083c       __IMPORT_DESCRIPTOR_api-ms-win-crt-string-l1-1-0 1000383c     ucrt:api-ms-win-crt-string-l1-1-0.dll
 0002:00000850       __IMPORT_DESCRIPTOR_api-ms-win-crt-heap-l1-1-0 10003850     ucrt:api-ms-win-crt-heap-l1-1-0.dll
 0002:00000864       __IMPORT_DESCRIPTOR_api-ms-win-crt-runtime-l1-1-0 10003864     ucrt:api-ms-win-crt-runtime-l1-1-0.dll
 0002:00000878       __IMPORT_DESCRIPTOR_api-ms-win-crt-convert-l1-1-0 10003878     ucrt:api-ms-win-crt-convert-l1-1-0.dll
 0002:0000088c       __NULL_IMPORT_DESCRIPTOR   1000388c     kernel32:KERNEL32.dll
 0003:00000000       ___security_cookie_complement 10004000     MSVCRT:gs_cookie.obj
 0003:00000004       ___security_cookie         10004004     MSVCRT:gs_cookie.obj
 0003:00000008       ___scrt_native_dllmain_reason 10004008     MSVCRT:utility.obj
 0003:00000010       ___isa_enabled             10004010     MSVCRT:cpu_disp.obj
 0003:00000014       ___scrt_ucrt_dll_is_in_use 10004014     MSVCRT:ucrt_stubs.obj
 0003:00000340       ?__type_info_root_node@@3U__type_info_node@@A 10004340     MSVCRT:tncleanup.obj
 0003:00000348       ?_OptionsStorage@?1??__local_stdio_scanf_options@@9@4_KA 10004348     MSVCRT:default_local_stdio_options.obj
 0003:00000350       ___scrt_current_native_startup_state 10004350     MSVCRT:utility.obj
 0003:00000354       ___scrt_native_startup_lock 10004354     MSVCRT:utility.obj
 0003:00000374       ___scrt_debugger_hook_flag 10004374     MSVCRT:utility_desktop.obj
 0003:00000378       ___isa_available           10004378     MSVCRT:cpu_disp.obj
 0003:0000037c       ___favor                   1000437c     MSVCRT:cpu_disp.obj
 0003:00000380       ?_OptionsStorage@?1??__local_stdio_printf_options@@9@9 10004380     <common>
 0003:00000388       ___dyn_tls_init_callback   10004388     <common>

 entry point at        0001:00000d5e

 Static symbols

 0000:ffff9000       .debug$S                   10000000     npt.exp
 0000:ffff9000       .debug$S                   10000000     vcruntime:VCRUNTIME140.dll
 0000:ffff9000       .debug$S                   10000000     vcruntime:VCRUNTIME140.dll
 0000:ffff9000       .debug$S                   10000000     vcruntime:VCRUNTIME140.dll
 0000:ffff9000       .debug$S                   10000000     vcruntime:VCRUNTIME140.dll
 0000:ffff9000       .debug$S                   10000000     vcruntime:VCRUNTIME140.dll
 0000:ffff9000       .debug$S                   10000000     ucrt:api-ms-win-crt-convert-l1-1-0.dll
 0000:ffff9000       .debug$S                   10000000     ucrt:api-ms-win-crt-heap-l1-1-0.dll
 0000:ffff9000       .debug$S                   10000000     ucrt:api-ms-win-crt-heap-l1-1-0.dll
 0000:ffff9000       .debug$S                   10000000     ucrt:api-ms-win-crt-heap-l1-1-0.dll
 0000:ffff9000       .debug$S                   10000000     ucrt:api-ms-win-crt-runtime-l1-1-0.dll
 0000:ffff9000       .debug$S                   10000000     ucrt:api-ms-win-crt-runtime-l1-1-0.dll
 0000:ffff9000       .debug$S                   10000000     ucrt:api-ms-win-crt-runtime-l1-1-0.dll
 0000:ffff9000       .debug$S                   10000000     ucrt:api-ms-win-crt-runtime-l1-1-0.dll
 0000:ffff9000       .debug$S                   10000000     ucrt:api-ms-win-crt-runtime-l1-1-0.dll
 0000:ffff9000       .debug$S                   10000000     ucrt:api-ms-win-crt-runtime-l1-1-0.dll
 0000:ffff9000       .debug$S                   10000000     ucrt:api-ms-win-crt-runtime-l1-1-0.dll
 0000:ffff9000       .debug$S                   10000000     ucrt:api-ms-win-crt-runtime-l1-1-0.dll
 0000:ffff9000       .debug$S                   10000000     ucrt:api-ms-win-crt-runtime-l1-1-0.dll
 0000:ffff9000       .debug$S                   10000000     ucrt:api-ms-win-crt-runtime-l1-1-0.dll
 0000:ffff9000       .debug$S                   10000000     ucrt:api-ms-win-crt-runtime-l1-1-0.dll
 0000:ffff9000       .debug$S                   10000000     ucrt:api-ms-win-crt-runtime-l1-1-0.dll
 0000:ffff9000       .debug$S                   10000000     ucrt:api-ms-win-crt-runtime-l1-1-0.dll
 0000:ffff9000       .debug$S                   10000000     ucrt:api-ms-win-crt-runtime-l1-1-0.dll
 0000:ffff9000       .debug$S                   10000000     ucrt:api-ms-win-crt-stdio-l1-1-0.dll
 0000:ffff9000       .debug$S                   10000000     ucrt:api-ms-win-crt-stdio-l1-1-0.dll
 0000:ffff9000       .debug$S                   10000000     ucrt:api-ms-win-crt-string-l1-1-0.dll
 0000:ffff9000       .debug$S                   10000000     ucrt:api-ms-win-crt-string-l1-1-0.dll
 0000:ffff9000       .debug$S                   10000000     kernel32:KERNEL32.dll
 0000:ffff9000       .debug$S                   10000000     kernel32:KERNEL32.dll
 0000:ffff9000       .debug$S                   10000000     kernel32:KERNEL32.dll
 0000:ffff9000       .debug$S                   10000000     kernel32:KERNEL32.dll
 0000:ffff9000       .debug$S                   10000000     kernel32:KERNEL32.dll
 0000:ffff9000       .debug$S                   10000000     kernel32:KERNEL32.dll
 0000:ffff9000       .debug$S                   10000000     kernel32:KERNEL32.dll
 0000:ffff9000       .debug$S                   10000000     kernel32:KERNEL32.dll
 0000:ffff9000       .debug$S                   10000000     kernel32:KERNEL32.dll
 0000:ffff9000       .debug$S                   10000000     kernel32:KERNEL32.dll
 0000:ffff9000       .debug$S                   10000000     kernel32:KERNEL32.dll
 0000:ffff9000       .debug$S                   10000000     kernel32:KERNEL32.dll
 0000:ffff9000       .debug$S                   10000000     kernel32:KERNEL32.dll
 0000:ffff9000       .debug$S                   10000000     kernel32:KERNEL32.dll
 0000:ffff9000       .debug$S                   10000000     kernel32:KERNEL32.dll
 0000:ffff9000       .debug$S                   10000000     kernel32:KERNEL32.dll
 0000:ffff9000       .debug$S                   10000000     kernel32:KERNEL32.dll
 0000:ffff9000       .debug$S                   10000000     kernel32:KERNEL32.dll
 0000:ffff9000       .debug$S                   10000000     kernel32:KERNEL32.dll
 0001:00000803       _getWideString             10001803 f   utf_md.obj
 0001:00000a1e       ?dllmain_crt_dispatch@@YGHQAUHINSTANCE__@@KQAX@Z 10001a1e f   MSVCRT:dll_dllmain.obj
 0001:00000a71       ?dllmain_crt_process_attach@@YAHQAUHINSTANCE__@@QAX@Z 10001a71 f   MSVCRT:dll_dllmain.obj
 0001:00000b78       ?dllmain_crt_process_detach@@YAH_N@Z 10001b78 f   MSVCRT:dll_dllmain.obj
 0001:00000c28       ?dllmain_dispatch@@YAHQAUHINSTANCE__@@KQAX@Z 10001c28 f   MSVCRT:dll_dllmain.obj
 0001:00000d33       ?dllmain_raw@@YGHQAUHINSTANCE__@@KQAX@Z 10001d33 f   MSVCRT:dll_dllmain.obj
 0001:00000ea3       ___get_entropy             10001ea3 f   MSVCRT:gs_support.obj
 0001:00000f98       ?find_pe_section@@YAPAU_IMAGE_SECTION_HEADER@@QAEI@Z 10001f98 f   MSVCRT:utility.obj
 0001:00001400       $$000000                   10002400     MSVCRT:sehprolg4.obj
 0002:00000290       _GS_ExceptionPointers      10003290     MSVCRT:gs_report.obj
 0002:00000718       __sehtable$?dllmain_crt_process_attach@@YAHQAUHINSTANCE__@@QAX@Z 10003718     MSVCRT:dll_dllmain.obj
 0002:00000738       __sehtable$?dllmain_crt_process_detach@@YAH_N@Z 10003738     MSVCRT:dll_dllmain.obj
 0002:00000760       __sehtable$?dllmain_dispatch@@YAHQAUHINSTANCE__@@KQAX@Z 10003760     MSVCRT:dll_dllmain.obj
 0002:00000780       __sehtable$___scrt_is_nonwritable_in_current_image 10003780     MSVCRT:utility.obj
 0002:000007a0       .edata                     100037a0     npt.exp
 0002:000007c8       rgpv                       100037c8     npt.exp
 0002:000007d0       rgszName                   100037d0     npt.exp
 0002:000007d8       rgwOrd                     100037d8     npt.exp
 0002:000007dc       szName                     100037dc     npt.exp
 0002:000007e4       $N00001                    100037e4     npt.exp
 0002:000007f2       $N00002                    100037f2     npt.exp
 0002:00000ad6       .idata$6                   10003ad6     kernel32:KERNEL32.dll
 0002:00000b28       .idata$6                   10003b28     vcruntime:VCRUNTIME140.dll
 0002:00000c54       .idata$6                   10003c54     ucrt:api-ms-win-crt-stdio-l1-1-0.dll
 0002:00000c74       .idata$6                   10003c74     ucrt:api-ms-win-crt-string-l1-1-0.dll
 0002:00000c96       .idata$6                   10003c96     ucrt:api-ms-win-crt-heap-l1-1-0.dll
 0002:00000cb6       .idata$6                   10003cb6     ucrt:api-ms-win-crt-runtime-l1-1-0.dll
 0002:00000cd8       .idata$6                   10003cd8     ucrt:api-ms-win-crt-convert-l1-1-0.dll
 0003:00000018       ?__proc_attached@@3HA      10004018     MSVCRT:dll_dllmain.obj
 0003:00000020       _GS_ExceptionRecord        10004020     MSVCRT:gs_report.obj
 0003:00000070       _GS_ContextRecord          10004070     MSVCRT:gs_report.obj
 0003:00000358       ?is_initialized_as_dll@@3_NA 10004358     MSVCRT:utility.obj
 0003:00000359       ?module_local_atexit_table_initialized@@3_NA 10004359     MSVCRT:utility.obj
 0003:0000035c       ?module_local_atexit_table@@3U_onexit_table_t@@A 1000435c     MSVCRT:utility.obj
 0003:00000368       ?module_local_at_quick_exit_table@@3U_onexit_table_t@@A 10004368     MSVCRT:utility.obj
 0004:00000060       $R000000                   10005060     npt.dll.res
